:100000000C947D010C94C4010C94C4010C94C401A3
:100010000C94C4010C94C4010C94C4010C94C4014C
:100020000C94C4010C94C4010C94C4010C94931E50
:100030000C944F1E0C94621F0C94C4010C94C401C8
:100040000C94C4010C94C4010C94C4010C943E1F84
:100050000C94C4010C94C4010C94C4010C94C4010C
:100060000C94C4010C94C4010C94C4010C94C401FC
:100070000C94C401C55CC45C000000007B007C00E3
:100080007D0000004B004E00A900AA0000001E00E9
:100090001F00200000010101010101010101020214
:1000A0000202020202020203030303030303030426
:1000B00004040404040405050505050606060606F1
:1000C000070707070708080808090909090A0A0AAB
:1000D0000B0B0B0C0C0C0D0D0D0E0E0E0F0F0F104D
:1000E00010111111121213131414151516161717D7
:1000F000181819191A1A1B1B1C1D1D1E1E1F202043
:10010000212222232424252626272829292A2B2C8C
:100110002D2D2E2F30313232333435363738393AAF
:100120003B3C3D3E3F404142434445464748494AA7
:100130004C4D4E4F50515354555658595A5B5D5E75
:100140005F616264656668696B6C6D6F7072737510
:1001500077787A7B7D7E8082838587888A8C8E8F74
:1001600091939596989A9C9EA0A2A3A5A7A9ABADA2
:10017000AFB1B3B5B7BABCBEC0C2C4C6C9CBCDCF90
:10018000D1D4D6D8DBDDDFE2E4E7E9EBEEF0F3F53E
:10019000F8FAFDFF05010902A10185020901A1008C
:1001A0000509190129081500250195087501810225
:1001B0000501093009311581257F950275088106F1
:1001C00009381581257F950175088106050C0A38C7
:1001D000021581257F950175088106C0C0050109BA
:1001E00080A101850319012AB700150126B70095E2
:1001F0000175108100C0050C0901A10185041901D8
:100200002AA002150126A002950175108100C005E3
:10021000010906A1018506050719E029E715002552
:10022000019508750181020507190029EF150025C0
:100230000195F075018102050819012905950575DB
:10024000019102950175039101C005010906A10103
:10025000050719E029E715002501950875018102B8
:100260009501750881010507190029FF150026FF72
:100270000095067508810005081901290595057581
:10028000019102950175039101C009023B00020131
:1002900000A0FA0904000001030101000921110175
:1002A00000012240000705810308000A090401003B
:1002B000010300000009211101000122B600070519
:1002C000820320000A12010002000000082D737052
:1002D0000C01000102000110033000780043002EE1
:1002E0000070006100640000000A0373002D006FBD
:1002F000006C000000040309040011241FBECFEFAE
:10030000D4E0DEBFCDBF04B603FE27C08091E50276
:100310009091E602A091E702B091E8028730904BFD
:10032000A740B04BD1F41092E5021092E602109271
:10033000E7021092E80214BE84B7877F84BF0FB62D
:10034000F894A89580916000886180936000109275
:1003500060000FBEE0E0F8E3099522E0AEE8B1E00E
:1003600001C01D92A53EB207E1F711E0A0E0B1E0A7
:10037000E2E9F8E402C005900D92AE38B107D9F772
:100380000E94891F0C9410240C9400009091DF02AD
:10039000937061F081110BC094609093DF02109212
:1003A00012018091DE0281608093DE020895833124
:1003B00010F09864F2CF880F880F982BEECF9091B1
:1003C000DF02937059F08093E0026093E102409362
:1003D000E2028091DE0281608093DE020895209126
:1003E000E4003091E50095E6A9012091EC00822F10
:1003F000817020FF06C08091E80080FF06C080E089
:1004000008952091E80022FD1AC08091A40288235B
:1004100089F0853089F08091EB0085FD0FC0209137
:10042000E4003091E50042175307F9F29150E1F6EC
:1004300084E0089582E0089583E0089581E00895BE
:10044000EF92FF920F931F93CF937C018B010E9439
:10045000EF01C82F811117C08091E80085FD0BC006
:100460008091E8008E778093E8000E94EF01882356
:1004700099F3C82F08C0F70181917F018093F100A3
:100480000150110949F78C2FCF911F910F91FF90C7
:10049000EF9008958091A60287FF13C08091E80035
:1004A00082FF06C08091E8008B778093E80004C04B
:1004B0008091A4028111F2CF08958091A402882333
:1004C000D9F38091E80080FFF8CF8091E8008E7723
:1004D000ECCF982F9093E900242F762F50E08917C6
:1004E00031F07091EC002091ED005091F00021FD71
:1004F00007C09F5F953071F78093E90081E0089510
:100500003091EB003E7F3093EB003091ED003D7F6A
:100510003093ED003091EB0031603093EB0070933D
:10052000EC002093ED005093F0002091EE0027FDA9
:10053000E0CF80E00895FC018091AC029091AD0283
:1005400086179707A0F06115710529F49091E800CE
:100550009E779093E80090E06115710551F4911138
:1005600008C08091E80082FF32C080E00895BC019D
:10057000F2CF8091A4028823B1F18530B1F180914E
:10058000E80083FD2EC08091E80082FDEACF8091D3
:10059000E80080FFE1CF2091F20030E061157105A5
:1005A00019F02830310558F091E02830310509F074
:1005B00090E02091E8002E772093E800CDCF819144
:1005C0008093F100615071092F5F3F4FE7CF809119
:1005D000A402882341F0853041F08091E80083FF38
:1005E000C0CF81E0089582E0089583E008950895E2
:1005F0008091810208959C014FB7F8948091770211
:1006000090917802A0917902B0917A024FBF821B3B
:10061000930B08952FB7F894809177029091780208
:10062000A0917902B0917A022FBF089520910E0116
:100630002223C9F020917B0227FF15C0E62FE69503
:10064000E695E695EE31D8F4E80FF92FF11D6770C5
:1006500021E030E001C0220F6A95EAF720958281FF
:10066000282322830895FC01329608962191621373
:1006700003C0DF0111971C92E817F907B9F7089535
:1006800020910E012223C1F020917B0227FF14C08C
:10069000E62FE695E695E695EE31F8F4E80FF92FAA
:1006A000F11D677021E030E001C0220F6A95EAF782
:1006B0008281822B82830895FC0132962FEF30E0F5
:1006C0004191641751F02F3F19F4411101C0232FBC
:1006D0003F5F3630A9F72F3F09F40895820F911D2F
:1006E00027FD9A95FC016283089520917402309150
:1006F00075022817390771F0909375028093740280
:10070000E0917202F0917302309721F00084F1853C
:10071000E02D0994089520917002309171022817FC
:10072000390771F09093710280937002E091720228
:10073000F0917302309721F00680F781E02D099443
:100740000895E0917202F0917302309721F00190C8
:10075000F081E02D099480E00895FA01811101C033
:10076000FB010994ECE4F2E08183608342833396D9
:1007700092E0E037F907C1F70895362F63E070E0A3
:100780000E942423DC01A45BBD4F11963C9311977A
:100790004C93FD0122830895EFEDF2E0248130E1D6
:1007A000231B08F420E024838091DE028160809383
:1007B000DE020895EFEDF2E0248130E1230F08F42A
:1007C0002FEF24838091DE0281608093DE02089502
:1007D000EFEDF2E0438120E1421B08F440E081812B
:1007E000628190E00C94DF01EFEDF2E0438120E1C3
:1007F000420F08F44FEF8181628190E00C94DF0199
:10080000EFEDF2E0628120E1621B08F460E081819B
:10081000438190E00C94DF01EFEDF2E0628120E192
:10082000620F08F46FEF8181438190E00C94DF0147
:10083000EFEDF2E08181438162818850990B0C9445
:10084000DF01EFEDF2E0818190E043816281089663
:100850000C94DF018091DF0286958695815009F422
:1008600082E10C94C6018091DF02869586958F5FA8
:10087000833108F081E00C94C601362F842F90E07C
:1008800066E070E00E942423820F911D70E0803C9E
:1008900050F48295869586958370E82FF0E0E95AAA
:1008A000FE4F30817FEF632F8FEF0895EF92FF921D
:1008B0000F939701201B31092F3F310519F010F0DC
:1008C0002FEF30E0322F3095482F430F08F44FEFD1
:1008D000842F620F0F91FF90EF900895EF92FF9297
:1008E0000F93E62F472F382F802F90E065E070E0C0
:1008F0000E9424238E0D9F1D8F3F910519F010F04B
:100900008FEF90E0282F2095320F08F43FEF6E2FE5
:10091000742F832F0F91FF90EF90089522E8241BEE
:1009200008F420E0620F0895362F272F4095682F96
:1009300070E0842F90E00E942423632F722F892F70
:100940000895362FB72FA82FE42FF0E0EE0FFF1FEA
:10095000E659FE4F8081821B87FD819590E068E11A
:1009600070E00E942423692F630F7B2F8A2F089544
:10097000EF920F93372F282F802F90E063E070E0E5
:100980000E942423959587956E2D680F732F822FD3
:100990000F91EF900895E42FF0E0EE0FFF1FE65A5D
:1009A000FE4F6189621B0895E42FF0E0EE0FFF1FF8
:1009B000E659FE4F6081621B0895622F0895CF9320
:1009C000DF93D62FC72FA82FB0E0E42FF0E0EE0F73
:1009D000FF1FE659FE4F808190E064EE70E00E94B8
:1009E0002423492F50E0445E5F4FCA01821B9109C6
:1009F0009C0197FF03C031952195310983E0220FB7
:100A0000331F8A95E1F7CD01821B930B97FF02C03C
:100A100090E080E0BD010E9424236D2F7C2F892F60
:100A2000DF91CF910895CF93C62F382FA72FB0E035
:100A3000E42FF0E0EE0FFF1FE659FE4F808190E0BB
:100A400064EE70E00E942423492F50E0CA014C96C6
:100A5000821B910997FF03C091958195910923E02D
:100A6000880F991F2A95E1F7AD01481B590BCA0160
:100A700057FF02C090E080E0BD010E9424236C2F4C
:100A8000792F832FCF9108950C94B2030C94BD035A
:100A9000FC019B01009729F480E077FF2BC080E8E0
:100AA0000895AC0197FF04C044275527481B590BF4
:100AB000B901640F751F37FD10C0241B350BC90128
:100AC000A5E0880F991FAA95E1F70E94492380E2CB
:100AD000861BF7FF0FC081950895CB0165E0880F55
:100AE000991F6A95E1F7BA01621B730B0E944923B3
:100AF00080E6EECF0895EF920F93CF93DF93D72F39
:100B0000C82FC9010E19BA010E944805602F681B41
:100B10007D2F8C2FDF91CF910F91EF900895EF9261
:100B20000F931F93CF93DF93162FD72FC82FC90191
:100B30000E190C0FBA010E944805081B6C2F70E0BB
:100B4000802F90E00E942423612F7D2F892FDF9139
:100B5000CF911F910F91EF900895EF920F931F93F4
:100B6000CF93DF93162FC72FD82FC9010E19070F68
:100B7000BA010E944805081B6C2F70E0802F90E09E
:100B80000E942423612F792F8D2FDF91CF911F9108
:100B90000F91EF900895282F8074E22F26FDE095A5
:100BA0006E2F6F7081116F5FE695E695E695E670A2
:100BB000F0E0E15BFE4F818170E090E00E94242331
:100BC000AC0184E0559547958A95E1F78081840FC3
:100BD00027FD819580580895FC01A82F029710F1F8
:100BE0004FEFE13E8EE1F80738F4AF0195E05695FE
:100BF00047959A95E1F7485FB1E08B2F840F9927CD
:100C0000991F9C0135952795A22FC901B9010E9412
:100C10002423E817F90740F44FEF420F4B1768F70A
:100C2000AFEFAB0F8A2F08952F3FE1F3B1E0B20F82
:100C3000F5CFCF92DF92EF92FF920F931F93CF9356
:100C4000DF93E82FF0E0EC56FF4F71110FC0949145
:100C5000292FE92F692F7E2F822FDF91CF911F91AE
:100C60000F91FF90EF90DF90CF900895262F30E006
:100C7000C72FD0E0E4914E2FEE2EF12CC90166E093
:100C800070E00E9424230FEF10E0B8010E9435238A
:100C9000DB01220F331FCB0165E570E00E942423A6
:100CA000281B390BC22ECC0CC20EC8018C1B9D0B0D
:100CB000B7010E942423292FD12CC601BE010E9416
:100CC0002423692F70E0C801861B970BB7010E948F
:100CD0002423392FC8018C199D09BE010E942423A9
:100CE000692F70E0C801861B970BB7010E9424236F
:100CF000892FA230B10589F040F4109709F4AACFEA
:100D0000119779F0922F232FA5CFA430B10561F070
:100D100078F0169709F49ECFF5CF9E2FE22F282F5B
:100D200099CF9E2FE32F96CF922F2E2FE82F92CF81
:100D3000E22F242F932F8ECFDF92EF92FF920F930B
:100D40001F93CF93DF937C0180910F01C82FCC0FAD
:100D5000C80F13E01C0F012F1D3008F00CE020918C
:100D6000E3022695269531E0230F08F42FEF6091DA
:100D7000D7027091D802822F90E00E942423D92EAE
:100D8000D0E0C01760F081E01C3008F080E0DF9117
:100D9000CF911F910F91FF90EF90DF900895FE018A
:100DA000E65AFE4F80A590911001892391F0609141
:100DB000E0027091E1028091E2022D2D4C2FF701AB
:100DC00009950E941906462F282F672FCE010E94F1
:100DD00046052196D6CF2F923F925F926F927F92D7
:100DE0008F929F92AF92BF92CF92DF92EF92FF923B
:100DF0000F931F93CF93DF93CDB7DEB72A970FB62C
:100E0000F894DEBF0FBECDBF8B837E836D83809150
:100E10000F01282F220F280F2F832D5F29832A836C
:100E20002D3010F03CE03A838091AE028C83FF813C
:100E3000EF2FF0E0FA87E987CF01880F991F9C0117
:100E4000265A3E4F69013B81832F90E0FC01319689
:100E5000F887EF838A8199859817E8F081E0E98126
:100E6000EC3008F080E02A960FB6F894DEBF0FBE93
:100E7000CDBFDF91CF911F910F91FF90EF90DF9049
:100E8000CF90BF90AF909F908F907F906F905F902A
:100E90003F902F900895E985FA85E65AFE4F80A588
:100EA00090911001892301F12090E0023090E1023D
:100EB0002F81388522553D4F39015B8010E0FC8140
:100EC0005F16E0F08091E202612F70E090E00E94F6
:100ED0002423B101892F0E941906462F282F672F3E
:100EE00089859A850E94460529853A852F5F3F4F5F
:100EF0003A87298732E0C30ED11CACCFF301819130
:100F00003F01F601A088A81ABB088188F3018781F8
:100F1000881A9908C501B5010E9424239C01C401C7
:100F2000B4010E942423820F931F0E94EC05082F16
:100F30002091E30231E0230F08F42FEFF301EE0FCD
:100F4000FF1FEE5AF24065897689822F90E00E9459
:100F50002423E92EF12C9401A501B101812FED810B
:100F6000FE8109951B015394182FA9CFCF92DF92D0
:100F7000EF92FF920F931F93CF93DF938C01809199
:100F80000F01C82FCC0FC80F53E0D52EDC0ECD2C8F
:100F90002CE02D1510F44CE0C42E2091E30231E03A
:100FA000230F08F42FEF30E050E040E06FEF7FEFC9
:100FB00080E090E00E94CF237901D0E02C2FCC1567
:100FC00070F081E0FBE0FD1508F480E0DF91CF9147
:100FD0001F910F91FF90EF90DF90CF900895FE0149
:100FE000E65AFE4F80A590911001892329F1809146
:100FF000AE028150082E000C990B87FF1FC0B7016D
:101000003091E30221E0320F08F43FEF832F90E0AC
:101010000E9424236091E0027091E1028091E2023B
:10102000492F50E0F80109950E941906462F282FF4
:10103000672FCE010E9446052196C0CFFC01E255E4
:10104000FD4F318932130AC0FC01EE0FFF1FE2553C
:10105000FD4F618D728D6E157F0590F20197CDCF9A
:101060005F926F927F928F929F92AF92BF92CF9238
:10107000DF92EF92FF920F931F93CF93DF933C0188
:1010800080910F01C82FCC0FC80F13E01C0FF12E59
:101090001D3010F03CE0F32E8091E30286956091C4
:1010A000D7027091D80290E00E942423592ED0E0FC
:1010B000CE01880F991F9C01265A3E4F6901CF151A
:1010C000A0F081E01C3008F080E0DF91CF911F910B
:1010D0000F91FF90EF90DF90CF90BF90AF909F90D7
:1010E0008F907F906F905F900895FE01E65AFE4FBB
:1010F00080A590911001892361F1F6018089282F44
:101100002057330B59018189E82FEF53FF0B4F0113
:10111000C901B9010E9424239C01CF01BF010E9493
:101120002423820F931F0E94EC05082F6091E00298
:101130007091E1028091E202E52C9401A501F30196
:1011400009950E941906462F282F672FCE010E946D
:101150004605F2E0CF0ED11C2196B1CF0E940A03C2
:101160009C0190911B0280911C02982B21F03093DE
:1011700018022093170290911D0280911E02982B55
:1011800021F03093160220931502E0917202F09143
:101190007302309749F082E0809319020480F58150
:1011A000E02D89E192E00994089540911B028D3E63
:1011B00059F480911C0287FF0DC010921C0241114E
:1011C0000BC01092130208C08E3E81F480911C0265
:1011D00018169CF3442381F080911D0290911E0209
:1011E000892B09F05AC01092120208958F3E49F4DB
:1011F00047FFF0CF10921B0280911C028111ECCFAF
:10120000E0CF803F19F41416ACF3E4CF90911D02A7
:10121000893F29F41916F4F610921D02DBCF8A3F9C
:1012200019F497FFD7CFF8CF90911E028B3F29F486
:1012300097FFD0CF10921E02CDCF8C3F19F4191614
:10124000CCF3C8CF9FE0980F983090F4815F990B52
:1012500021E030E0B90102C0660F771F8A95E2F7FE
:10126000CB01809590911A02892380931A02B2CF04
:101270008D3F31F4809114028E7F80931402AACFA7
:101280008E3F21F4809114028D7FF7CF8F3F09F0BC
:10129000A1CF809114028B7FF0CF0895809114022A
:1012A00080FD18C081FD18C082FD18C08091120217
:1012B0008823B1F0883290F490E023E0880F991FE2
:1012C0002A95E1F768E270E00E944923862F672B98
:1012D00039F0089582E0089584E0089588E0089543
:1012E00081E008958091140280FD15C081FD15C034
:1012F00082FD17C080911302882389F0843188F41D
:1013000090E062E370E00E94242364E170E00E94B8
:101310004923862F08958CE0089589E1089585E09A
:10132000089582E308958D3E31F40E9472098195FB
:1013300080931C0208958E3E19F40E947209F8CF22
:101340008F3E31F40E947209819580931B020895AB
:10135000803F19F40E947209F8CF893F29F40E9456
:101360004E0980931D0208958A3F21F40E944E0980
:101370008195F7CF8B3F31F40E944E098195809380
:101380001E0208958C3F19F40E944E09F8CF9FE089
:10139000980F983070F4815F990B21E030E001C024
:1013A000220F8A95EAF780911A02822B80931A0203
:1013B00008958D3F31F4809114028160809314026E
:1013C00008958E3F21F4809114028260F7CF8F3F01
:1013D000B9F7809114028460F1CF80E00895F89409
:1013E000E82FE295EF70F0E031A1282F2F7081E017
:1013F00090E001C0880F2A95EAF7982F90959323E3
:1014000091A392A1892B82A37894089590917B0255
:1014100092FF06C0282F28712830F9F4877F846056
:1014200093FF06C0282F28712831F1F4877E84614C
:1014300020917C0220FF06C0382F38713830D9F453
:10144000877F816021FF06C0282F28712831D1F4C1
:10145000877E816194FD877E0895282F2471243032
:10146000F9F68B7F8860DCCF282F2471243101F7B7
:101470008B7E8861DDCF382F3171313019F78E7F47
:101480008860E0CF282F2171213121F78E7E88617D
:10149000E1CFCF93DF93EC0182389105A9F1D8F524
:1014A0008133910509F496C048F58932910509F414
:1014B0008AC08A9709F495C0C11521E5D20708F0C2
:1014C000BCC0C11530E5D30708F016C1C83ED10530
:1014D00008F09CC0C03ED10560F5C83AD10508F0BF
:1014E00087C0C53AD10508F0FFC0C130D10509F168
:1014F0002097F9F0C430D105E0F440C08533910560
:1015000009F45AC0C997C1F680917B02837089F0B3
:10151000C0EED0E00EC0833E910599F170F4803E9C
:10152000910501F1823E910539F680917B0282FDA1
:1015300021C0CE01DF91CF910895863E910561F1E2
:10154000873E910571F1843E910509F0B5CF8091F8
:101550007C0281FFEECF80917B02C7EED0E084FD5C
:101560000DC0E7CF80917B0280FD18C190917C0275
:1015700090FFDFCFC3EED0E084FFDBCFD0E0C0E050
:10158000D8CF80917B0282FD0CC190917C0290FDAE
:10159000BFCF84FFCECFF2CF80917B0283FDDDCF22
:1015A000C8CF80917B0283FDFFC090917C0291FFA8
:1015B000F0CFC4EED0E0BDCF80917B0285FFB9CFE4
:1015C000C9E2D0E0B6CF80917B0285FFB2CFC5E300
:1015D000D0E0AFCF80917B0286FFABCFCAE2D0E0F4
:1015E000A8CF80917B0286FFA4CFC1E3D0E0A1CF3A
:1015F000CF3BD10518F6C85AD0E0CC0FDD1FC75E2F
:10160000DE4F0990D881C02DD46493CFC11540E23C
:10161000D40758F4C11581E0D80708F08ACFCD3E31
:10162000D10508F4ABCFD06584CFC11520E4D20733
:1016300008F4A4CFDF70D06A7CCFC11535E5D3079D
:1016400010F5C11544E5D40708F090C0C11583E535
:10165000D80708F075C0C11522E5D20708F46BC0A1
:10166000CE018370992721E030E002C0220F331FA2
:101670008A95E2F7C695C695D0E0E5E0CC0FDD1F70
:10168000EA95E1F754C0C11539E5D307A8F4C115AF
:1016900048E5D40708F06FC0C11586E5D80708F003
:1016A0006DCF8C2F0E94060AC82FD0E0DC2FCC27EC
:1016B000CC27DF71D0623DCFC1152AE5D20708F4EF
:1016C0005FC0CE0190568115904208F057CF8D2F04
:1016D0008F710E94060A90E0982F882788279F71B3
:1016E0009C012C2BE901E6CFC55AD0E0CA5EDE4F43
:1016F000C881D0E0D0641DCFCE01A4E09695879537
:10170000AA95E1F783702C2F26952695237030E05B
:10171000B5E0220F331FBA95E1F7382B8C2F837079
:10172000C1E0D0E002C0CC0FDD1F8A95E2F7C22BEA
:10173000D32BDC68FECEDC2FCC27C16FD06AF9CE6C
:10174000CE018370992721E030E002C0220F331FC1
:101750008A95E2F7C695C695D0E075E0CC0FDD1FFF
:101760007A95E1F7C22BD32BDA68E3CEDC2FCC27B6
:10177000C46FD06ADECEDC2FCC27C06FD06AD9CE42
:101780008C2F8F700E94060A34E0D695C7953A9543
:10179000E1F7CF709C2FEC01D069CBCEC9E3D0E04C
:1017A000C8CEC2EED0E0C5CEC6EED0E0C2CE8091AB
:1017B000F70181111092F701089580959091F6013B
:1017C00098239093F60108958091F6019091F50188
:1017D000892B9091F401892B809390019091F701CE
:1017E0009923A1F0892B8093900180910E01882389
:1017F00041F180917B0287FF24C08EE1E2E9F1E0B4
:1018000090E0815000F591110E94D70BE091720297
:10181000F09173023097E1F080910E01882359F026
:1018200080917B0287FF07C0809190018093910196
:1018300086E0809390010280F381E02D80E991E0C1
:10184000099486E0DBCF21912223D9F29F5FD9CF83
:1018500008958091F2019091C101981301C00895FB
:101860008F5F8770FACF8F929F92AF92BF92DF9275
:10187000EF92FF920F931F93CF93DF93809000021C
:1018800090900102A0900202B09003024091F801F2
:101890005091F9016091FA017091FB01842A952A17
:1018A000A62AB72ACFE1D0E0E92EF12C082F10E0CC
:1018B000DC2ED501C4010C2E04C0B695A7959795D2
:1018C00087950A94D2F780FD10C0219788F7D12C14
:1018D0008D2DDF91CF911F910F91FF90EF90DF90B1
:1018E000BF90AF909F908F900895FE01EE0FFF1F65
:1018F000EE0FFF1FEE0DFF1DEE0FFF1FEE0FFF1F80
:10190000E00FF11FEE0FFF1FEC58FF4F85919491F0
:101910000E94490A0197C9F2DBCFCF93DF93EC0114
:101920000E94330CE82FF0E0EE0FFF1FEE0FFF1FB9
:10193000ED0FF11DEE0FFF1FEE0FFF1FEC0FF11D5E
:10194000EE0FFF1FEC58FF4F85919491DF91CF91DF
:101950000C94490A990F990F890FA82FA7708695A3
:101960008695869590E065E070E00E942423FC0156
:10197000EF54FE4F50E040E080E0219130E00A2E2D
:1019800002C0369527950A94E2F721703327042E7A
:1019900001C0220F0A94EAF7822B4F5F5F4F453058
:1019A000510559F70895CF93DF93262F990F990F7B
:1019B000890F982F9770E1E001C0EE0F9A95EAF732
:1019C00086958695869590E065E070E00E942423D8
:1019D000DC01AF54BE4F50E040E0622F70E08D91CB
:1019E000ED0121979B01042E02C0369527950A949C
:1019F000E2F72170219528272E23282728834F5F7F
:101A00005F4F4530510559F7DF91CF910895FC01A3
:101A1000808191810E948D0C292F2F7092959F704B
:101A200092509E3078F4E92FF0E0EE5EFB4D0C947E
:101A30005D23803F19F020F4883E20F481E0089572
:101A4000843FE1F380E00895883EC0F3813FD1F701
:101A5000F5CF822F869586958695089590E080E053
:101A60000E948B0390E080E00E9475031092F501C4
:101A70001092F4010E94E40B86E0E9E1F2E0DF015C
:101A80001D928A95E9F71092130210921202109299
:101A900014020C94AE0860930002709301028093CC
:101AA0000202909303020C942E0D0F931F9341E0BA
:101AB00050E060E070E004C0440F551F661F771FC0
:101AC0008A95D2F7CB01BA01609570958095909573
:101AD0000091000210910102209102023091030254
:101AE00060237123822393231F910F910C944B0D3C
:101AF0009091F301809589238093F301282F27701B
:101B000091F4282F082E000C330B9217130659F06E
:101B100090917C0292FD07C08595859585950E94E0
:101B2000550D1092F30108950F931F9341E050E07B
:101B300060E070E004C0440F551F661F771F8A9550
:101B4000D2F78091000290910102A0910202B0911F
:101B500003028A019B01082B192B2A2B3B2BC9015D
:101B6000B8011F910F910C944B0D6093F801709385
:101B7000F9018093FA019093FB010C942E0D8823B8
:101B800021F00E94DD0B0C94E40B0895882339F0BA
:101B90009091F601982B9093F6010C94E40B089524
:101BA000882379F19CEF980F913A38F4682F80E9F7
:101BB00091E00E9416030C94E40B90E2980F983089
:101BC00050F4877091E001C0990F8A95EAF7892F48
:101BD0000E94DD0BF0CF9BE5980F933020F490E04E
:101BE00080E00C948B0398E5980F973120F490E0F7
:101BF00080E00C9475038D3E20F00E94D5080C9473
:101C0000AE080895CF93C82F882309F46FC08CEFD6
:101C10008C0F813AC0F580910E01882311F18091DB
:101C20007B0287FF1EC0EC2FE695E695E695F0E077
:101C3000E057FE4F828190E04C2F477021E030E06A
:101C400002C0220F331F4A95E2F782239323892B88
:101C500091F06C2F80E991E00E9416030E94E40B42
:101C60000AC0E2E9F1E088E991E02191C21789F325
:101C70008E179F07D1F76C2F80E991E00E944003F7
:101C8000CF910C94E40B80E28C0F883068F4C7701D
:101C900021E030E001C0220FCA95EAF78091F601F9
:101CA000822B8093F601ECCFEBE5EC0FE33040F4B0
:101CB000F0E0EA5EFE4F808190E0CF910C948B03C0
:101CC000E8E5EC0FE73150F4F0E0EE0FFF1FE75EC0
:101CD000FE4F80819181CF910C947503CD3E30F001
:101CE0008C2F0E949309CF910C94AE08CF91089548
:101CF0000F931F93CF93DF93C62FD42F022FFC0196
:101D000082818823A1F06093DD020E940A039093F0
:101D1000DC028093DB02C77081E001C0880FCA95A6
:101D2000EAF7DF91CF911F910F910C94C60D80912E
:101D3000DD02681338C08091DB029091DC020E94C2
:101D4000FB02883C910578F510E21D0FCD17B9F024
:101D500080E28C0F883040F4C77081E001C0880FAA
:101D6000CA95EAF70E94BF0D183048F481E09D2F14
:101D7000977001C0880F9A95EAF70E94C60D802FD0
:101D80000E94020E802F0E94D00D183098F4D77058
:101D900081E001C0880FDA95EAF7DF91CF911F91BA
:101DA0000F910C94BF0DC77081E001C0880FCA95D8
:101DB000EAF7F3CFDF91CF911F910F9108958093B0
:101DC0007D0270937F0260937E028091A402843032
:101DD00001F582E08093E9008FEF9091E800815057
:101DE00095FD06C095ED9A95F1F700008111F5CFAC
:101DF0008091E80085FF0DC050E040E063E070E0B6
:101E00008DE792E00E9420028091E8008E77809317
:101E1000E8000895BC0184E00C94DF0EBC0183E06F
:101E20000C94DF0E9C0182E08093E9009FEF80918B
:101E3000E800915085FD06C085ED8A95F1F7000018
:101E40009111F5CF8091E80085FF0CC050E040E093
:101E500066E070E0C9010E9420028091E8008E7760
:101E60008093E8000895CF93DF93EC0180910E01F9
:101E70008823B1F180917B0287FF32C060E282E06B
:101E80008093E9008FEF9091E800815095FD06C0A6
:101E900095ED9A95F1F700008111F5CF8091E8005A
:101EA00085FF1BC080910E0170E050E040E0811181
:101EB00004C050E040E068E070E0CE010E942002E3
:101EC0008091E8008E778093E80080E2FE01A2E82E
:101ED000B2E001900D928A95E1F7DF91CF910895DC
:101EE00068E081E0CDCF81E08093E00080E28093E4
:101EF000D8001092C9008FE19EE40197F1F700C06D
:101F0000000087E090EBDC018093E5029093E6020D
:101F1000A093E702B093E80288E19CE00FB6F89442
:101F2000A895809360000FBE90936000FFCF3F9A0A
:101F300038B13F7728B120684FB7F8948CE492E02D
:101F4000FC015191CF0168E028B9000000C057FFA3
:101F500038B9550F000000C000C000C038B900C03B
:101F60006A9591F7F2E080379F0751F74FBF8FE5F1
:101F700094E00197F1F700C0000008958F929F92BE
:101F8000AF92BF92CF92DF92EF92FF920F931F9387
:101F9000CF93DF938091480290914902A0914A0229
:101FA000B0914B022FB7F89480907702909078020E
:101FB000A0907902B0907A022FBF75016401C81A0F
:101FC000D90AEA0AFB0A2FB7F89440917702509198
:101FD00078026091790270917A022FBF4093480293
:101FE0005093490260934A0270934B0210911F0272
:101FF000EFE1F2E0C12FD0E00197AF4FBF4F88195A
:102000009909AA09BB091D1324C0C0931F0280911E
:10201000DF02182F137019F0182F1695169590914E
:102020001201913009F43FC0992331F1923009F443
:1020300080C1933009F485C1DF91CF911F910F9139
:10204000FF90EF90DF90CF90BF90AF909F908F90D8
:102050000895218D328D4901B12CA12C8815990547
:10206000AA05BB0520F4C150DF5F3296CCCF2C0D02
:102070003D1D328F218FF8CF10920F014093D70270
:102080005093D8026093D9027093DA0289E2EFE1AB
:10209000F2E0AEEAB2E001900D928A95E1F781E0BC
:1020A00080931201C9CF90910D01191322C0837042
:1020B00020910C0130E091E08217130609F490E0C2
:1020C000892F8170809311018091E4029091100119
:1020D000981739F08093100140E060E080E00E94A2
:1020E0004405133190F4E12FF0E0E05EFB4D0C94D9
:1020F0005D2381E0E6CF80911101882309F488C037
:1021000040E060E080E00E94440580E081C0809172
:102110000F01C82FCC0FC80F03E00C0FF02E0D30AD
:1021200010F02CE0F22E6091E0027091E1028091BB
:10213000E2020E941906E62ED72EC82ED0E0CF1557
:1021400028F081E00C3008F463C0DFCFFE01E65ACE
:10215000FE4F80A590911001892331F02C2D4E2D3A
:102160006D2DCE010E9446052196E9CF80910F0189
:10217000C82FCC0FC80F03E00C0FF02E0D3010F05D
:102180009CE0F92ED090E002E090E102D091E202D2
:102190008091E3028695869586956091D70270912D
:1021A000D80290E00E942423892F0E94CB058058FA
:1021B00087FD8195880F6D2F70E090E00E942423A9
:1021C0006D2D7E2D892F0E941906E62ED72EC82E42
:1021D000D0E0CF1508F0B5CFFE01E65AFE4F80A53E
:1021E00090911001892331F02C2D4E2D6D2DCE01B3
:1021F0000E9446052196EDCF83E195E00E949C0662
:1022000007C08FED94E0FACF8DEA95E00E94300888
:1022100090910F019F5F90930F0181110DCF82E08C
:102220008093120180911101811106CF111104CF09
:1022300083E036CF8FE895E0E9CF8DED94E0DECFF7
:1022400084ED94E0DBCF8BEC94E0D8CF88EB94E086
:10225000DDCF8BE795E0DACF80910F01C82FCC0F4F
:10226000C80F03E00C0FF02E0D3010F08CE0F82EAC
:10227000D090E102E090E202D091E0028091E3028E
:102280008695869586956091D7027091D80290E0E8
:102290000E942423892F0E94CB05805887FD8195B9
:1022A000880F90E06CE070E00E9424236D2F690F8E
:1022B0007D2D8E2D0E941906E62ED72EC82ED0E039
:1022C000CF1508F03ECFFE01E65AFE4F80A5909153
:1022D0001001892331F02C2D4E2D6D2DCE010E9441
:1022E00046052196EDCF81EA94E088CF84E994E019
:1022F0000E94B6078DCF8EE894E0FACF8091AE02AF
:1023000021E0382F321B08F430E0832F6EE674E0B2
:102310000E94EB067DCF8091AE0221E0382F321B68
:1023200008F430E0832F66E574E0F2CF8DE394E0AB
:1023300065CF10930D01837080930C010E94970F5D
:1023400077CF8091DE02882351F046E050E06CE1C7
:1023500070E08FED92E00E949B231092DE0240918C
:10236000D7025091D8026091D9027091DA022FB74A
:10237000F8948091770290917802A0917902B091BF
:102380007A022FBF841B950BA60BB70B4097A105B4
:10239000B10508F451CE109212014ECEEFEDF2E0ED
:1023A00089E480838091130190911401A09115011B
:1023B00081839283A3838FE784838FEF858346E0B5
:1023C00050E06CE170E0CF010E949B231092DE028E
:1023D00008951092F60180910E01E2E9F1E0882360
:1023E00059F080917B0287FF07C08EE1DF011D92CB
:1023F0008A95E9F70C942E0D86E0F8CF1F93CF93C2
:10240000DF93CDB7DEB7AA970FB6F894DEBF0FBE45
:10241000CDBF86EA92E02091F100FC012193CF012B
:10242000F2E08E3A9F07B9F78091A702833009F452
:102430006EC0B8F4813009F445C0823009F4AFC0F1
:102440008091E80083FF7BC28091A6029091A70251
:102450009A3008F074C2E92FF0E0ED5CFB4D0C946B
:102460005D238A3009F48AC08B3009F46DC089304D
:1024700039F78091A602813219F78091AA029091D2
:10248000AB020297E8F68091E800877F8093E8002E
:102490008091E80082FF36C08091F200823031F4F2
:1024A0008091F100813011F0863021F48091F100AB
:1024B000809381028091E8008B778093E8000E94EE
:1024C0004A02BECF8091A602813A09F0B9CF80912D
:1024D000E800877F8093E8008091AA029091AB0288
:1024E000892B61F460E282E892E070E00E949B0236
:1024F0008091E8008B778093E800A2CF60E090E0C5
:1025000080E0F3CF8091A4028111C2CF99CF809156
:10251000A602813A09F094CF8091AA029091AB0271
:10252000892B09F08DCF8091E800877F8093E800A8
:102530008091E80080FFFCCF80910E018093F10034
:102540008091E8008E77B9CF8091A602813209F0A0
:1025500077CF8091AA029091AB02892B09F070CFBE
:102560008091E800877F8093E8000E944A02809172
:10257000A80280930E010E94E91162CF8091A60209
:10258000813209F05DCF8091E800877F8093E80079
:102590000E944A028091A9028093800251CF8091CB
:1025A000A602813A09F04CCF8091E800877F8093A2
:1025B000E8008091E80080FFFCCF80918002BECFD0
:1025C000803899F0823809F0BAC18091AA028F70E0
:1025D000853008F0B4C18093E9008091EB0085FB61
:1025E000882780F91092E90006C08091A20290919C
:1025F000A302911182609091E800977F9093E80088
:102600008093F1001092F1008091E8008E7793C1E1
:10261000882309F481C1823009F091C18091A80218
:10262000811184C18091AA028F702FEF280F24306E
:1026300008F085C18093E9002091EB0020FF76C16E
:10264000933031F48091EB0080628093EB006EC197
:102650009091EB0090619093EB0021E030E001C09D
:10266000220F8A95EAF72093EA001092EA008091FF
:10267000EB008860EACF811162C11091A8021F7738
:102680008091E3008078812B8093E3008091E800C3
:10269000877F8093E8000E944A028091E80080FFD3
:1026A000FCCF8091E30080688093E30082E0111109
:1026B00083E08093A40243C18058823008F03FC178
:1026C0008091A8029091A9028C3D23E09207A1F588
:1026D00083E08A838AE289834FB7F894DE011396F8
:1026E00020E03EE051E2E32FF0E050935700E49108
:1026F00020FF03C0E295EF703F5FEF708E2F90E0F8
:10270000EA30C0F0C7968D939D932F5F243159F71F
:102710004FBF8091E800877F8093E8006AE270E015
:10272000CE0101960E949B028091E8008B778093F6
:10273000E80005C1C096E7CF4091AA025091AB02D4
:10274000292F33272330310509F444C078F521308F
:10275000310509F46FC08BE390E0EAE8F2E0223043
:10276000310509F0ECC02091E800277F2093E800B4
:102770002091AC023091AD028217930708F49C01BE
:1027800040E02115310509F064C0411162C080911B
:10279000E80082FDC9CF8091A402882329F2853008
:1027A00019F28091E80083FFF2CFBECF21323105CC
:1027B000A9F12232310509F0C2C04115510509F4D1
:1027C00043C04130510509F0BAC086EB90E0E4E91E
:1027D000F1E0C9CF992781309105C1F0009759F0F8
:1027E000029709F0ACC0E7EDF2E0E4918E2F90E0A3
:1027F000E7EDF2E007C0E5EFF2E0E4918E2F90E024
:10280000E5EFF2E0009709F49AC0ADCFE9EEF2E00F
:10281000E4918E2F90E0E9EEF2E0F4CF41155105FE
:1028200071F04130510509F08AC089E090E0E5EB94
:10283000F2E099CF82E190E0E5ECF2E094CF89E01C
:1028400090E0ECE9F2E08FCF80E490E0EAE4F2E09F
:102850008ACF8091A402882309F466CF853009F4D9
:1028600063CF8091E80083FD5FCF8091E80082FD17
:102870008ECF8091E80080FF84CF8091F20090E0BD
:102880002115310519F08830910550F041E0089785
:1028900009F040E08091E8008E778093E80071CFE6
:1028A00044914093F1003196215031090196E8CFCF
:1028B000803809F044C08091E800877F8093E80069
:1028C0008091A5028093F1009FCE811138C01091B4
:1028D000A8021230A0F58091E800877F8093E8007D
:1028E0001093A5020E944A02112311F084E005C052
:1028F0008091E30087FDFACF81E08093A40242E05B
:1029000061EC81E00E94690242E261EC82E00E9497
:1029100069028091A40213C08091A802813079F4E9
:1029200081E0933009F080E08093A3021092E900E7
:102930008091E800877F8093E8000E944A0280919E
:10294000E80083FF0AC08091E800877F8093E80059
:102950008091EB0080628093EB00AA960FB6F8940A
:10296000DEBF0FBECDBFDF91CF911F910895CF93F2
:1029700084E090E00E948D23C82F82E290E00E94C4
:102980008D23982F8C2FCF9108958F929F92BF9275
:10299000CF92DF92EF92FF920F931F93CF93DF932B
:1029A00000D000D0CDB7DEB719821A821B821C82FC
:1029B00007E411E09BE4E92E91E0F92EBB24B394E7
:1029C000CC24C394D12CF80181918F018F3F09F45D
:1029D0004AC0F894E82FE295EF70F0E021A18F70E3
:1029E000A60102C0440F551F8A95E2F7CA01922F33
:1029F000982B91A392A18095892382A3789400C0FB
:102A00008BE4882E81E0982EDE0111966B2D609567
:102A1000F40191914F018D919D01215031099F3F0A
:102A200009F465C0492F42954F7050E0FA0140A16A
:102A300050E09F7002C0559547959A95E2F740FD8A
:102A400056C08B29F9018083FFE48F16F1E09F06C1
:102A5000F9F6F801319780818F3F11F00E94EF095C
:102A600040EA4A95F1F7BB0CE016F10609F0ABCF4E
:102A700044E050E0BE016F5F7F4F84E092E00E942F
:102A8000632311E0009709F410E0892B91F189810B
:102A90009A81AB81BC818093040290930502A0933C
:102AA0000602B093070281E08093FE010E940A03B0
:102AB0009093FD018093FC018091FC019091FD01B8
:102AC0000E94FB020597C8F08091040280930802DF
:102AD00080910502809309028091060280930A0288
:102AE0008091070280930B021092FE0106C086239C
:102AF000A9CF8091FE018111DFCF812F0F900F9020
:102B00000F900F90DF91CF911F910F91FF90EF9059
:102B1000DF90CF90BF909F908F90089569EE7EEFE9
:102B200090E080E00E94C92360E082E090E00E9493
:102B3000AB2360E083E090E00E94AB231092F801A9
:102B40001092F9011092FA011092FB0160E084E00A
:102B500090E00E94AB2360E082E290E00E94AB2311
:102B600060E085E090E00E94AB2360E086E090E0CA
:102B70000E94AB236FEF87E090E00E94AB2340E020
:102B800050E0BA0188E090E00E94BD2360E08DE053
:102B900090E00E94AB2340E050E0BA0188E190E071
:102BA0000E94BD2360E087E190E00E94AB2340E0FB
:102BB00050E0BA018CE190E00E94BD2370E060E03B
:102BC00080E290E00E94C92340E050E0BA0188E131
:102BD00090E00E94BD2340E050E0BA018FE090E019
:102BE0000E94BD2340E050E0BA0183E190E00C94E4
:102BF000BD23CF93C0917C02C2FB992790F998170F
:102C000099F080FBC2F9C0937C0260917B0284E062
:102C100090E00E94AB236C2F82E290E00E94AB23F5
:102C200082E0CF910C94780DCF9108954F925F92EE
:102C30006F927F928F929F92AF92BF92CF92DF92CC
:102C4000EF92FF920F931F93CF93DF9300D000D0AA
:102C50000F92CDB7DEB77C01FC0183819481892B73
:102C600039F0D08011818D2D81238F3F09F0CDC4A3
:102C70000F900F900F900F900F90DF91CF911F91B9
:102C80000F91FF90EF90DF90CF90BF90AF909F900B
:102C90008F907F906F905F904F9008950E94330CBB
:102CA000082F682F89819A810E94D30CE02FF0E0D1
:102CB000EE0FFF1FEE0FFF1FE10FF11DEE0FFF1FC5
:102CC000EE0FFF1FED0DF11DEE0FFF1FEC58FF4F34
:102CD00005911491043FFCE51F0709F498C0D0F555
:102CE000093D3CE5130709F48EC00A3D8CE5180741
:102CF00009F49DC0083D9CE51907C1F526E241EEA7
:102D000061EEC7010E94780E8091F301877009F48B
:102D1000AFCFF7018281882309F4AACF80917C028A
:102D200082FDA6CF82E00F900F900F900F900F9032
:102D3000DF91CF911F910F91FF90EF90DF90CF9097
:102D4000BF90AF909F908F907F906F905F904F90CB
:102D50000C94780D063FECE51E0709F460C008F4FA
:102D60005AC0073F2CE5120709F45DC0F7018281C4
:102D7000882309F45BC41092DD020430FDE51F07CF
:102D800008F058C00B3F2CE5120730F4C801825000
:102D90009C45449708F053C00E94B71490937C025E
:102DA00080937B0200318CE5180709F41BC108F001
:102DB00097C00830ECE51E0709F402C108F069C0AD
:102DC00004302CE5120709F4EDC008F04FC00230C2
:102DD0008CE5180709F4E0C080917B028260033023
:102DE0001C4509F4DCC060917B0210917C0284E0F8
:102DF00090E00E94AB23612F82E290E00E94AB231F
:102E00000E94E91181CF27E245EE65EE7ACF26E2F6
:102E100041EE60EE76CF27E245EE64EE72CF26E219
:102E200041EE62EE6ECF27E245EE66EE6ACF28E213
:102E300041E0EBCF02363DE5130709F4ADCF8091B9
:102E4000F6010631ECE51E0709F0FDC38A7A91E030
:102E500009F490E09093B00169E2811165E380E9A3
:102E600091E00E9440030E94E40B4ECF80917B02D0
:102E700080610630ECE51E0709F491C080917B0269
:102E8000886007301C4508F48AC080917B0280620C
:102E900086C080917B028D7F0C302CE5120709F4EF
:102EA0007EC058F40A308CE5180709F493C008F482
:102EB0008BC080917B028E7F72C080917B02877F66
:102EC0000E30ECE51E0709F46AC080917B028B7F0F
:102ED0000F301C4508F463C080917B028F7E5FC079
:102EE0000D3F2CE5120709F479C068F504318CE533
:102EF000180709F48BC080F40231ECE51E0709F4D1
:102F000075C080917B028F7B03311C4508F447C05C
:102F100080917B02837F43C00B3F2CE5120709F4AD
:102F200045C008F049C005311C4509F05CCF8091CF
:102F30007B0282FB992790F921E0922790FB82F98E
:102F400090FB83F92CC001309DE5190709F454C0AA
:102F500088F480917C0283600F3FFCE51F0749F1F4
:102F600080917C028D7F01151D4518F180917C02B6
:102F70008C7F1FC003303DE5130709F456C008F4E9
:102F80004EC002361D4509F02ECF90917B02892F4D
:102F90008F7E94FF806103C080917B02816080936B
:102FA0007B0221CF80917B028460F9CF80917C02EB
:102FB000816080937C0217CF80917C028260F9CF80
:102FC00080917B028064EBCF0E94E91180917B02AB
:102FD0008068E5CF80917B028C60E1CF80917C029C
:102FE0008E7FE7CF80917B028F7DD9CF0E94E91140
:102FF00080917B028F77D3CF80917C02982F909520
:1030000091708E7F892B90FB81F9D3CF0E94E911BB
:1030100090917B02892F97FB87F98058C0CF61E0A0
:103020008EE090E00E94AB23DECE60E0F9CF80918D
:10303000DF0291E089278093DF02109212018091D4
:10304000DE0281608093DE025FCE4AE254E063E3F9
:1030500074E00E94AD0358CE43E354E06AE274E0AA
:10306000F8CF48E154E061E274E0F3CF41E254E08C
:1030700068E174E0EECF40E054E06CE074E0E9CF4A
:103080004CE054E060E074E0E4CF44EF53E068EEDD
:1030900073E0DFCF4AED53E06CEC73E0DACF82E00F
:1030A00081C30C359DE5190701F10D351D4509F06A
:1030B000F5C280917C0282FB882780F991E0892704
:1030C0000E94F915EBC20E94E911FFEF24E33CE0F6
:1030D000F15020403040E1F700C000000E94730F23
:1030E0000E948E1511CE81E0EBCF80E0E9CF812FD9
:1030F000902F0E94AA0CD82EE2C2212F2F70C22E30
:10310000107F19F0C29460EFC622DD20B9F0CC2008
:1031100069F080E2800F883010F0811009C0809142
:10312000F601C82AC092F6010E94E40B802F4BC022
:103130008091F501C82AC092F501F6CF802F0E9438
:10314000D00DCC2009F441C0005E083010F0811091
:1031500004C08C2D0E94DD0B06C0C0948091F50147
:10316000C822C092F5010E94E40B2FC0312F3F709E
:10317000C32E107F103219F0C29450EFC522882060
:1031800089F081E0881609F48BC0DD2009F495C030
:10319000992009F48BC0F701858180FFC7CF8F701C
:1031A000858384C020917C0222FF57C0DD2009F472
:1031B0004DC0CC2039F08091F601C82AC092F601AA
:1031C0000E94E40B80E00E94020EEA2DE850FF0B03
:1031D000349710F40E94A103BB20A9F08091F30161
:1031E00080FD11C0F70112828595859585950E9415
:1031F000940DC7010E9416168091F301859585955F
:1032000085950E94550D85E0F701DE01119601902C
:103210000D928A95E1F789819A810E94AA0C90E02B
:10322000880F991F880F991FEA818E0F911D880FB3
:10323000991F880F991FE981E80FF92FF11DEE0FF3
:10324000FF1FEC58FF4F8591949112CD80E00E94B2
:10325000D00DCC2009F4B9CF7CCFDD20A1F0909126
:10326000F7018C2D892B911003C00E94C60DADCFA4
:10327000E1E09E12FACF22FDA8CF981709F4A5CF5E
:103280008093F701A2CF911006C00E94D70B8C2D1E
:103290000E94BF0D9ACFF1E09F1609F496CFF5CFAB
:1032A000DD2031F025E0291508F48FCF8C2DDDCFFE
:1032B00034E0391508F489CFEACF992041F3F9E3D6
:1032C0008F1209C02FEF37EE83E02150304080404D
:1032D000E1F700C00000802F0E94D00D76CF812F33
:1032E00086958695837061F0813009F06ECFC801B4
:1032F0009370D11002C090E080E00E94750365CF0A
:10330000C8019370D11002C090E080E00E948B034E
:103310005CCF802FDD2029F00E9493090E94AE0827
:1033200054CF0E94D508FACF812F837009F066C070
:10333000D1104BCF802F829586958770880F880F8C
:10334000602F6F70462E512C712C612C082E04C0FA
:10335000440C551C661C771C0A94D2F740E050E0E0
:10336000BA0104FF0FC04FE050E060E070E004C01D
:10337000440F551F661F771F8A95D2F740955095C9
:1033800060957095812F869586958370823019F1AE
:10339000D8F40091F8011091F9012091FA013091CF
:1033A000FB01813069F04429552966297729CB0131
:1033B000BA0160237123822393230E94B50D05CFA8
:1033C000402A512A622A732ACB01BA01642975293D
:1033D00086299729F2CF4429552966297729009112
:1033E000F8011091F9012091FA013091FB01CB0114
:1033F000BA016027712782279327DFCF8695DD20CA
:1034000011F0812F8170882309F4DFCE802F8295FF
:1034100086958770880F880F602F6F70462E512C0D
:10342000712C612C082E04C0440C551C661C771CA2
:103430000A94D2F740E050E0BA0104FF0FC04FE019
:1034400050E060E070E004C0440F551F661F771F16
:103450008A95D2F74095509560957095812F869505
:1034600086958370823019F1D8F400910002109192
:1034700001022091020230910302813069F0442957
:10348000552966297729CB01BA016023712382234C
:1034900093230E944B0D99CE402A512A622A732A07
:1034A000CB01BA016429752986299729F2CF4429CD
:1034B0005529662977290091000210910102209177
:1034C000020230910302CB01BA01602771278227E3
:1034D0009327DFCF1F70DD2029F0812F0E94940DEC
:1034E000802FC3CE802F0E94BF0D812F0E94550DCB
:1034F0006CCE802F92EF891609F43FC0981570F0BA
:10350000E0EF8E16D1F0F1EF8F1691F0DD2009F487
:103510006CC091100BCE812F8F7133C023EF8216B8
:1035200099F134EF8312F2CF80917C0282FF3FC089
:10353000812F8F71DD20D1F224C0DD20C9F084E01D
:10354000891508F442CE1F7161E070E080E090E0E0
:1035500004C0660F771F881F991F1A95D2F7009134
:103560000002109101022091020230910302ADCFBE
:1035700095E0991508F429CEE6CF812F8F71D110EF
:10358000B5CF0E94940D21CE60E070E0CB01DD202C
:1035900009F47FCF1F7161E070E080E090E004C02B
:1035A000660F771F881F991F1A95D2F772CFDD20FB
:1035B00089F01F71812F0E94940D80917C0282FD01
:1035C00007C0812F880F880F880F83608093F301D5
:1035D000812FD7CF81E00E94780DE1E0E91508F056
:1035E000F4CD82E00E94780DF0CD992059F0893316
:1035F00009F071CEFFEF27EE33E0F150204030406C
:10360000E1F767CE812F8F7171CF85E0DE011196D2
:1036100001900D928A95E1F7F701228189819A81C3
:1036200021113CCB0E94AA0C082F40CB06311C452F
:10363000A9F58091B00169E2811165E380E991E02B
:103640000E94160310CC82720B3C2CE5120709F481
:103650001CCD08F093C0063C9CE5190709F401CD88
:1036600008F076C0043CFCE51F0709F4EECC08F036
:10367000F3CC033C3CE5130709F4D9CC0B35FDE54D
:103680001F0709F430CD08F00CCD01153CE51307F8
:1036900009F419CD0F3D1C4509F422CDF7018281B3
:1036A00010810181882309F422CD812F902F0E945F
:1036B000330CD82E682F812F902F0E94D30CED2D24
:1036C000F0E0EE0FFF1FEE0FFF1FE00FF11DEE0FFA
:1036D000FF1FEE0FFF1FE10FF11DEE0FFF1FEC5854
:1036E000FF4F859194910E94490A8C01882EF70121
:1036F000D280958092948FE098228091F301877018
:10370000C1F0BD2CDD20B1F0812F807F803421F00D
:1037100080E2800F883068F080917C0282FD09C0D1
:1037200082E00E94780D8091F3018770BB24B394EE
:103730008111B12CA12EA2947FE0A722FBE0FA1503
:1037400008F443CDEA2DF0E0E35CFB4D0C945D23DF
:10375000083C9CE5190709F48ECC08F487CC093C99
:10376000FCE51F0709F48CCC48EE53E064EF73E0EE
:103770000A3C2CE5120709F46CCC80CF0F3C3CE5E9
:10378000130709F48CCC88F40D3CECE51E0709F412
:1037900081CC4CEC53E06AED73E00E3C1C4508F420
:1037A00058CC81E00E94C601AFCA073D2CE5120744
:1037B00028F488E0013D1C45A8F3A6CA0E358DE526
:1037C000180709F4A1CA5ACF1F93CF93DF938091B2
:1037D000C001807FA1F48091BD01882381F02091F8
:1037E000F2011091C1014091BB01A091BC01C091B7
:1037F000BE01D091BF01B42FBA23121304C0DF91D0
:10380000CF911F91089530E0209711F0BF3F21F430
:103810002F5F3F4F2770F1CFC90166E070E00E9433
:103820002423FC01EE53FE4F81818A13F1CF808166
:103830008413EECF82818111EBCF838194818C1B25
:103840009D0B883C910520F78091C0018F708061AD
:103850008093C001C90166E070E00E942423FC014E
:10386000E953FE4F90819F70906190838BEB91E0C4
:103870000E941616DF91CF911F910C94290CAF92E4
:10388000BF92CF92DF92EF92FF920F931F93CF934D
:10389000DF93CDB7DEB761970FB6F894DEBF0FBEEA
:1038A000CDBF8C0185E0F801DE011D9601900D92DF
:1038B0008A95E1F7D8011296EC9012978BEBA82E1F
:1038C00081E0B82E6091BE017091BF016115710554
:1038D00009F438C19091BB012091BC01892F82234A
:1038E0008F3F09F42FC14C911196EC9111971396CB
:1038F000CD90DC90F090BD01D601A61BB70BFF2048
:1039000009F4EBC08091C001382F307FA83CB1058D
:1039100008F0AEC031117AC0FE2C2E1321C09413D2
:103920001FC0E1101DC08F7080618093C001C50170
:103930000E9416168091C001F80185838F2D619633
:103940000FB6F894DEBF0FBECDBFDF91CF911F91B0
:103950000F91FF90EF90DF90CF90BF90AF900895C0
:10396000CD2829F0842F8E238F3F09F006C180E0F7
:10397000F82FF170DF2E2091F201F091C10180FD4E
:1039800021C0EE20D9F28091C00181608093C001F6
:10399000F12CD4CF30E0C90166E070E00E9424230E
:1039A000DC01AE53BE4F11968C911197E81307C0FE
:1039B0008C91481304C012968C91E812E2CF2F5FCD
:1039C0003F4F27702F13E6CF4D87EE878D859E855D
:1039D0000E948D0C292F22952F70223058F0243010
:1039E00080F49F7059F0D80115969C91907F31F426
:1039F000D12C0AC09F7011F08823D1F3805E8830EB
:103A0000B8F3C8010E941616FD2C98CF2E1306C0DD
:103A1000941304C0F801EE2009F479C0C8010E9493
:103A2000070D882309F1EE20F9F08091C001803262
:103A300070F02091BB013091BC0138872F8319862B
:103A4000DB86CA868C87CE0107960E94161686E012
:103A5000F801ABEBB1E001900D928A95E1F70E947D
:103A6000E41BFF24F3946ACFC8010E941616F9CF15
:103A700031110AC08BEB91E00E94161686E0D50149
:103A80001D928A95E9F784CF2E130FC094130DC0B1
:103A9000E1100BC0F8018583C8010E94161686E06C
:103AA000D5011D928A95E9F749CFC8010E94070DFB
:103AB0008823D1F2EE20C1F28091C001803238F229
:103AC0002091BB013091BC013A8329831B82DD82A6
:103AD000CC828E83CE010196B8CFA83CB105F8F612
:103AE000FE2CEE2009F22E131FC094131DC08091EE
:103AF000C00180FD10C0982F907F69F0F801858388
:103B0000903F31F0982F907F905F8F70892B858345
:103B1000C8010E94161686E0F801ABEBB1E00190F7
:103B20000D928A95E1F70ACFC8010E94070D811115
:103B30008ECF8091C00181608093C001C8010E9436
:103B40001616FCCEEE2009F48FCFC8010E94070D97
:103B5000F82E882309F488CF86E0F801ABEBB1E0BA
:103B600001900D928A95E1F78091BB019091BC0183
:103B70000E948D0C0E94E41BE1CE81E08E25F8CEE0
:103B8000CF93DF93CDB7DEB767970FB6F894DEBF5C
:103B90000FBECDBF4B8B5C8B6D8B7E8B8F8B611182
:103BA0001092F5011A8A198A85E0FE017396DE01EA
:103BB0001D9601900D928A95E1F786E0FE013D96F3
:103BC000DE01179601900D928A95E1F7CE010796D6
:103BD0000E943F1C811112C086E0FE013796DE0173
:103BE000119601900D928A95E1F78A859B85892B24
:103BF00029F08F81988589238F3FB1F58091F2015B
:103C00009091C10189131CC067960FB6F894DEBF6E
:103C10000FBECDBFDF91CF91089566E070E00E94A6
:103C20002423DC01AE53BE4F96E0FE013196019095
:103C30000D929A95E1F72093C1010E94290CDECFE5
:103C400090E066E070E00E9424238E539E4F0E9415
:103C50003F1C8823C9F28091F20190E001968770A1
:103C600099278093F201CACF8091C10190E09C0115
:103C70002F5F3F4F277033274091F2014217130601
:103C800061F60E94E9111092C1011092F20186E0E2
:103C9000EBEBF1E0DF011D928A95E9F7AFCF1F92C0
:103CA0000F920FB60F9211242F933F934F935F9370
:103CB0006F937F938F939F93AF93BF93CF93DF9334
:103CC000EF93FF93D091E900DF708091EC00C82F53
:103CD000C17080FDC0E81092E9008091F000877FFC
:103CE0008093F00078940E94FE111092E900809178
:103CF000F00088608093F000CD2BCF70C093E90076
:103D0000FF91EF91DF91CF91BF91AF919F918F91F3
:103D10007F916F915F914F913F912F910F900FBEC7
:103D20000F901F9018951F920F920FB60F921124AB
:103D30002F933F934F935F936F937F938F939F93B3
:103D4000AF93BF93EF93FF938091E10082FF09C08F
:103D50008091E20082FF05C08091E1008B7F80931B
:103D6000E1008091E10080FF17C08091E20080FFB8
:103D700013C08091E2008E7F8093E2008091E20088
:103D800080618093E2008091D80080628093D800A7
:103D900019BC85E08093A4028091E10084FF2BC0D0
:103DA0008091E20084FF27C084E089BD86E089BD60
:103DB00089B5982F917080FFFBCF8091D8008F7DBF
:103DC0008093D8008091E1008F7E8093E100809104
:103DD000E2008F7E8093E2008091E2008160809318
:103DE000E2008091A502882309F441C084E0809319
:103DF000A4028091A4028091E10083FF27C08091FA
:103E0000E20083FF23C08091E100877F8093E1007F
:103E100082E08093A4021092A5028091E1008E7F3F
:103E20008093E1008091E2008E7F8093E200809198
:103E3000E20080618093E20042E060E080E00E9466
:103E400069028091F00088608093F000FF91EF910B
:103E5000BF91AF919F918F917F916F915F914F91A2
:103E60003F912F910F900FBE0F901F90189580914A
:103E7000E30087FD93E09093A402BBCF78941F9258
:103E80001FB61F9211248F939F93AF93BF9380917E
:103E9000770290917802A0917902B0917A0201960E
:103EA000A11DB11D8093770290937802A0937902AF
:103EB000B0937A02BF91AF919F918F911F901FBED7
:103EC0001F9018951F921FB61F9211248F939F93D6
:103ED000AF93BF9380917602811113C080917702D6
:103EE00090917802A0917902B0917A024196A11D39
:103EF000B11D8093770290937802A0937902B093DA
:103F00007A02BF91AF919F918F911F901FBE1F901A
:103F10001895CDB7DEB760970FB6F894DEBF0FBE29
:103F2000CDBF84B7877F84BF0FB6F894A8958091E2
:103F30006000886180936000109260000FBE80E88E
:103F400090E00FB6F89480936100909361000FBEEB
:103F50008DEE99E090938F0180938E011092E20094
:103F60001092E1008091E00081608093E0008091F8
:103F7000D8008F778093D80019BC8091630081604E
:103F8000809363001092FF01809163008E7F809385
:103F9000630081E08093FF011092E2001092E10043
:103FA0008091D8008F778093D8008091D800806866
:103FB0008093D8008091D8008F7D8093D80084E0D2
:103FC00089BD86E089BD89B5282F2170E22E80FF4A
:103FD000FACF1092A4021092A5021092A30210929E
:103FE000A20242E060E080E00E9469028091E1006C
:103FF0008E7F8093E1008091E20081608093E200F7
:104000008091E20088608093E2008091E0008E7FE2
:104010008093E0008091E20084608093E2007894D5
:104020008091A4028823A1F01091E9001F70909163
:10403000EC00892F817090FD80E8182B1092E90028
:104040008091E80083FD0E94FE111F701093E9002B
:1040500082E084BD93E095BD9AEF97BD80936E009A
:1040600084E90E94EF0983E90E94EF0982E90E9436
:10407000EF0981E90E94EF0987E30E94EF0986E3D7
:104080000E94EF0985E30E94EF0984E30E94EF0993
:1040900084E0E8E0F2E0DF01282F1D922A95E9F79D
:1040A000E4E0F2E0DF011D928A95E9F790E080E01C
:1040B0000E949523893E9E4F11F00E948E1582E04A
:1040C00090E00E948D2380930D020E94B71490937C
:1040D0007C0280937B020E94C5148FE39CE90197C8
:1040E000F1F700C000000E94C5148091080280FF13
:1040F00008C06FEF7FEF90E080E00E94C9230E942C
:10410000730F83E090E00E948D23682F70E090E0B1
:1041100080E00E94B50D1092AE028FEF9FEF90935A
:10412000C8028093C7029093CA028093C9029093F9
:10413000CC028093CB029093CE028093CD029093D9
:10414000D0028093CF029093D2028093D1029093B9
:10415000D4028093D3029093D6028093D50210921A
:104160001F02909339028093380290933B02809310
:104170003A0290933D0280933C0290933F028093D9
:104180003E029093410280934002909343028093B9
:104190004202909345028093440290934702809399
:1041A000460290E080E00E949523893E9E4F21F0D8
:1041B0000E948E150E94CE1146E050E06CE170E046
:1041C0008FED92E00E947D231092DE028091DF024B
:1041D0008C7F11F40E94CE1180E091E090937302E5
:1041E0008093720208E1C02ED12C88E092E094E026
:1041F000692E680E18E0A12EB12C8091A402B0E4C3
:10420000FB2E04E016E0853009F4AAC10E94C51413
:10421000882359F08FB7F894409177025091780233
:104220006091790270917A028FBFA8E0B2E0EEE06F
:10423000F2E010E000E0902FFD9081918F1509F4DD
:10424000B3C18F25912C8E2C282F282109F4A7C1CA
:104250009F829887F82081E009F480E089870E9496
:104260000A038160782F9B878A874F8158856985EB
:104270008B850E94C01DF801E25FFD4F808188267A
:104280008082FF2079F0F801EE0FFF1FEE0FFF1F75
:10429000E65AFE4FE90DF11D8081F12C8F3F11F0A0
:1042A000782EFE2C0F2D10E080911F02800F912F91
:1042B000911D09975CF14501801A910AB801605E71
:1042C0007D4FA40180E292E00E947223B801685DF4
:1042D0007D4FA40188E292E00E947223A401440F62
:1042E000551FB801660F771F685C7D4F88E392E029
:1042F0000E947223B801605D7D4FA40180E392E0CB
:104300000E94722388E08F1980931F0280911F0200
:1043100090E0A72DB0E09D01220F331F26593E4F9C
:10432000AA0FBB1FBD0165597E4F41E0480F9F1585
:1043300008F420C180931F020E94BE0F86E0E9E1CD
:10434000F2E0DE01119601900D928A95E1F7F0906E
:104350001B0290901C0210911D0200911E021092EF
:104360001B0210921C0210921D0210921E028F2D31
:10437000892909F44DC080911702909118020E947A
:10438000FB029C0190911302992309F44FC123333E
:10439000310508F43DC09F3F19F09F5F90931302D1
:1043A000FF2051F00E9472096FEF1F140CF46E2D64
:1043B0000E941B2380931B02992051F00E947209D6
:1043C0006FEF19140CF46E2D0E941B2380931C02B6
:1043D00080911B028823E1F020911C022223C1F06E
:1043E000082E000C990B65EB70E00E9424239923A2
:1043F00009F4F1C090931B02822F220F990B65EBF9
:1044000070E00E942423992309F4E9C090931C02D0
:10441000812F802B09F44DC08091150290911602D6
:104420000E94FB029C0190911202992309F4F9C0A9
:104430002536310508F43DC09F3F19F09F5F9093EA
:104440001202112351F00E944E096FEF11160CF465
:104450006E2D0E941B2380931D02002351F00E94A9
:104460004E096FEF10160CF46E2D0E941B238093E3
:104470001E0280911D028823E1F020911E0222235A
:10448000C1F0082E000C990B65EB70E00E9424230C
:10449000992309F4A8C090931D02822F220F990B33
:1044A00065EB70E00E942423992309F4A0C0909347
:1044B0001E0280911B0290911C02892B90911D027B
:1044C000892B90911E02892B11F00E94AE0886E084
:1044D000FE013196A9E1B2E001900D928A95E1F7D3
:1044E0000E94A10390910C02891709F486CE0E94C4
:1044F000A10380930C027ECE8091A402843019F136
:104500000E94BE0F109276020FB6F894A895C09242
:1045100060000FBEF092600083B7817F846083BF2C
:1045200083B7816083BF7894889583B78E7F83BF7C
:104530000FB6F894A8958091600088618093600020
:10454000109260000FBE8091A302882349F00E9460
:10455000C514E8E0F2E0819181114DC06E12FBCFED
:104560008091A402853009F4C7CF0E94E9110E940E
:10457000A1034CCE90E0FC01E15EFD4FD9015C91BE
:104580005183DB015C915187718A880F991FFC016F
:10459000E15EFD4F128E118E842F9E2DC6CE939418
:1045A000880C24E0921250CE0F5F1F4F043011058B
:1045B00009F041CE8FEF8C878D871E860E940A03FB
:1045C0008160782F988B8F874C855D856E85888973
:1045D0000E94C01DB1CE81E080931B020DCF81E00F
:1045E00080931C0215CF81E080931D0256CF81E09D
:1045F00080931E025ECF09BD19BD09B400FEFDCF38
:104600008091D8008F7D8093D8008091E0008260F7
:104610008093E0008091E00081FDFCCF0E94E911D1
:104620009FCF2D32314008F009CF43CF2D3231409A
:1046300008F0B3CEEDCE002480FD060E660F11F01B
:104640008695D1F7802D08950024552704C0080EC3
:10465000591F880F991F009729F076956795B8F331
:104660007105B9F7802D952F0895AA1BBB1B51E149
:1046700007C0AA1FBB1FA617B70710F0A61BB70BD2
:10468000881F991F5A95A9F780959095BC01CD0177
:10469000089597FB072E16F4009407D077FD09D0F4
:1046A0000E94352307FC05D03EF4909581959F4FDD
:1046B0000895709561957F4F0895EE0FFF1F059047
:1046C000F491E02D0994E62FF72FA82FB92F04C0FD
:1046D0008D910190801921F441505040C8F7881BFA
:1046E000990B0895E62FF72FA82FB92F02C001903C
:1046F0000D9241505040D8F70895DC01CB01FC01E8
:10470000F999FECF06C0F2BDE1BDF89A319600B42A
:104710000D9241505040B8F70895F999FECF92BDDF
:1047200081BDF89A992780B50895A8E1B0E042E0EC
:1047300050E00C947F23DC01A40FB51F4150504082
:1047400048F0CB01840F951F2E910E94AC2341505D
:104750005040D0F70895262FF999FECF92BD81BD24
:10476000F89A019700B4021639F01FBA20BD0FB6AF
:10477000F894FA9AF99A0FBE08950396272F0E948B
:10478000AC230E94AB23252F0E94AC23242F0C9432
:10479000AC230196272F0E94AC230C94AB23052E4B
:1047A00097FB1EF400940E94E62357FD07D00E9459
:1047B000EE2307FC03D04EF40C94E623509540956D
:1047C000309521953F4F4F4F5F4F089590958095BD
:1047D000709561957F4F8F4F9F4F0895A1E21A2EDC
:1047E000AA1BBB1BFD010DC0AA1FBB1FEE1FFF1F95
:1047F000A217B307E407F50720F0A21BB30BE40BE5
:10480000F50B661F771F881F991F1A9469F760952B
:104810007095809590959B01AC01BD01CF010895E5
:10482000F894FFCF190D190D220D220D240D220D24
:10483000220D220D190D190D290D220D220D290D04
:104840007B108710B610FC10011104111A111D11F4
:1048500020112311261129112C11731176117B11AE
:104860007E118B119611E01208139F1408139F14E8
:104870003B135C139F14581465147D187D18B618EB
:10488000B6186F198919E518E51894196A1A791A72
:02489000791A93
:10489200F802330F120F0E0F0A0FF702FFFF01008B
:1048A200FF000300FFFF818283E200E900EA00B516
:1048B20000B600B700CD008301CC008A01920194BA
:1048C200012102230224022502260227022A02B320
:1048D20000B4006F00700094939291373635340023
:1048E2003131295A1B750A0055AA0006000001053C
:1048F20007000204080B0003090A606E5053403798
:10490200501C60377053806E90538037701C901C1F
:0E491200A03704040404040404040404040490
:00000001FF
